:10000000000000308A004E280C1E042899000314BA
:100010004A28211904280800A300A2012308031775
:100020008D000313240803178F001F2003194A288B
:100030000920A30A0319A40AA20F0E284A2883162E
:1000400003178C170C140000000083120C084A28B8
:10005000A801A700FF30A707031CA807031C4A2814
:100060000330A600DF3036202A28A601E83EA5008E
:10007000A609FC30031C3F28A50703183C28A50748
:100080000000A60F3C2825184528A51C492800007B
:1000900049280800831383120313080083160630CF
:1000A000990020309800831290309800A0016430AD
:1000B0008A0128200430A1000030A4007E308A018B
:1000C0000C200A308A0104200D308A010420C83037
:1000D0008A0128200430A1000030A40086308A0163
:1000E0000C200A308A0104200D308A0104208A0184
:1000F0005A2863008A0179288A017C28520061000D
:100100006400690020003A00290000004E006500EC
:100110002000720061006400690020003A0028009D
:020120000000DD
:02400E00323F3F
:00000001FF
